:100000000208D17F3CDFFE22D2003202000890FEBF
:1000100082E030E6F9E054BFF0223202001A7B00A1
:100020007A0079217528037F02120066E521C45405
:100030000775F00AA4FFE521540F2FF508E522C447
:10004000540775F00AA4FFE522540F2FF512E5239B
:10005000C4540375F00AA4FFE523540F2FF51522AD
:100060003232320200601208791208DD7FA31208D2
:10007000B512088E120897EF120543740129F9E4AE
:100080003AFAE528640160031208C3D528E612088D
:08009000A61208E653BA7F2214
:03009B00020061FF
:1000A3000200627593007594005391CF5392CF75FC
:0C00B300CB0075CC0075E10075E2002266
:1000C30002044FAD07ED707EC28C1204FDFEC39493
:1000D300037480948040037FFF22E58954FC4EF52E
:1000E30089900001120516FED39402748094804017
:1000F300037FFF22EEFF7E007006538E7F5389FB42
:10010300EF64014E7006438E805389FBEF64024E09
:100113007003438904900002120516FFE58F54FE15
:100123004FF58F900003120555E5F0F58C90000311
:10013300120555F58A9000051205167004C28C80CD
:1001430002D28C7F0022ED640160030201D6C28ECD
:100153001204FDFEC394037480948040037FFF2246
:10016300EEC454F0FFE58954CF4FF5899000011296
:100173000516FED394027480948040037FFF22EE21
:10018300FF7E007006538EBF5389BFEF64014E702C
:1001930006438E405389BFEF64024E700343894088
:1001A30090000212051625E0FFE58F54FD4FF58FF1
:1001B300900003120555E5F0F58D900003120555E7
:1001C300F58B9000051205167004C28E8002D28E44
:1001D3007F0022ED64027061538EEF9000011205DF
:1001E30016FF7E007006538EFB538EF7EF64014EAD
:1001F3007006438E04538EF7EF64024E7003438EF2
:100203000890000212051625E025E0FFE58F54FB58
:100213004FF58F900003120555E5F0F5D6900003D6
:10022300120555F5D7900005120516C454F0FFE5E5
:100233008E54EF4FF58E7F0022ED6403706953D126
:10024300F7900001120516FED39402748094804047
:10025300037FFF22EEFF7E00700653D1FD53D1FBD7
:10026300EF64014E700643D10253D1FBEF64024E9B
:10027300700343D104900002120516FFE5D154FE2A
:100283004FF5D1900003120555E5F0F5D490000326
:10029300120555F5D590000512051633333354F87E
:1002A300FFE5D154F78076ED6404707753D17F90E6
:1002B3000001120516FD7C00D394027480948040E3
:1002C300037FFF22ED4C700653D1DF53D1BF900063
:1002D300011205166401700643D12053D1BF90006B
:1002E300011205166402700343D140900002120507
:1002F30016C454F0FFE5D154EF4FF5D1900003122B
:100303000555FDACF0ECF5D2AF058FD39000051287
:100313000516C43333335480FFE5D1547F4FF5D1F1
:100323007F00227FFF221200A6120838120859D23A
:10033300AFE4F51BFFEFC3940874809480500974F5
:100343000A2FF876100F80ED12001EC2D5C3E50800
:10035300943C748094804002D2D5C3E512943C74DB
:100363008094804002D2D5C3E5159418748094809C
:100373004002D2D530D50BE4F508F51275150C12F1
:1003830006F512078F750C11750F11E4F518F513A7
:10039300F514F517F516F5093000FDC2001207D65E
:1003A300051AE51A70020519C394E8E51994034088
:1003B3000BE4F519F51A12001E12078F0509C3E5A0
:1003C300099432748094804006E4F509120610AF54
:1003D30013EF60C4641170160515C3E51594187402
:1003E3008094804003E4F5151206F512078FE51398
:1003F300641270161515C3E5159418748094804023
:10040300037515171206F512078FE5136413701899
:10041300F5080512C3E512943C748094804003E40C
:10042300F5121206F512078FE51364147018F50818
:100433001512C3E512943C74809480400375123BFB
:100443001206F512078FE4F51302039BC0E0C08385
:10045300C082C0D075D000C005C006C007AFBA4384
:10046300BA8090FE84E030E606E054BFF0807A90D4
:10047300FE84E030E535E054DFF0E51D6005751DD1
:10048300008066E51C600D751C0090FE87E0F51E7C
:100493002400803490FE87E0FEAD1E051E74002DFF
:1004A300F582E43400F583EEF0803E90FE84E03084
:1004B300E424E054EFF0E030E10890FE8674FFF0AE
:1004C3008027051E7400251EF582E43400F583E0C1
:1004D30090FE86F0801390FE84E030E30CE054F746
:1004E300F0751D01751C01D2018FBAD007D006D05B
:1004F30005D0D0D082D083D0E032BB010689828A76
:1005030083E0225002E722BBFE02E32289828A8330
:10051300E49322BB010CE58229F582E5833AF58356
:10052300E0225006E92582F8E622BBFE06E9258291
:10053300F8E222E58229F582E5833AF583E4932202
:10054300BB010689828A83F0225002F722BBFE0197
:10055300F322BB0110E58229F582E5833AF583E0B6
:10056300F5F0A3E0225009E92582F886F008E62297
:10057300BBFE0AE92582F8E2F5F008E222E5832AC8
:10058300F583E993F5F0A3E9932243BA809000023F
:100593001205166401702990FE80E04440F090FE3D
:1005A30082E4F01204FD543FFF90FE80E054C04FFC
:1005B300F0900003120516640190FE88702C8030C1
:1005C30090FE80E054BFF090FE84E4F090000412AB
:1005D300051625E0FF90FE85E054014FF0900005DD
:1005E300120516640190FE857006E054FEF0800447
:1005F300E04401F090000112051690FE807006E0C1
:10060300547FF08004E04480F053BA7F22AE177524
:1006130080F0120003E58054F0F51775800F120087
:1006230003E580540F42176317FFEE65177050AE52
:1006330014851714E5146044C2D5EE7004D2D58036
:1006430016EEB514120516E516C39414748094803F
:100653004005751612D2D530D525E514C4540F9034
:10066300092293FE6019E514540F93FF6011EE25E0
:10067300E025E0FEEF2E240CF5138003E4F5167558
:1006830080FF22EFD394017480948040037FFF2284
:1006930043BA80EF64017012ED90FE817006E0545E
:1006A3007FF08011E04480F0800BEF700890FE83B0
:1006B300E054874DF0EBFF7E00D394037480948065
:1006C300502DEF700653B6DF53B5DFEF64014E7064
:1006D3000653B6DF43B520EF64024E700643B620DF
:1006E30053B5DFEF64034E700643B62043B5207F56
:1006F3000022E50875F00A84C454F0FFE50875F09C
:100703000A84E5F02FF521E51275F00A84C454F04C
:10071300FFE51275F00A84E5F02FF522E51575F073
:100723000A84C454F0FFE51575F00A84E5F02FF54B
:10073300237B007A0079217528037F0202080DEFDD
:10074300FBD39401748094805009EB7004C2A98098
:1007530002D2A9EDFF7E00D39403748094805029C4
:10076300EF700553B7FDC2B9EF64014E700553B77F
:10077300FDD2B9EF64024E700543B702C2B9EF640C
:10078300034E700543B702D2B97F0022C3E5159427
:100793000A74809480400AE51575F00A84F50A808E
:1007A30003750A10E51575F00A8485F00B750C11B5
:1007B300E51275F00A84F50DE51275F00A8485F0EB
:1007C3000EE50875F00A84F510E50875F00A8485CE
:1007D300F01122C37407951BFFE49400FE741A2FD3
:1007E300F58274093EF583E493F4F5F8740A251B46
:1007F300F8E69008EF93F4F5E8051BC3E51B9408AE
:10080300748094804003E4F51B228B258A26892774
:10081300120879AB250527E527AA267002052614B9
:10082300F91204FDFF1208B512088ED528E5120847
:10083300E653BA7F22E4F521752201F5237524A23C
:10084300752540752601FB7A007921FF1200C6E465
:10085300FD7F01020742752301752201E4F524752A
:100863002110FB7A00792112058DE4FBFD7F011233
:10087300068653BACF22AE0743BA801208DD7FA2A1
:100883001208B512088EAF061208B590FE817403E4
:10089300F002000E90FE817404F012000E90FE87A9
:1008A300E0FF2290FE827401F090FE817405F00255
:1008B300000E90FE86EFF090FE817402F002000EAF
:1008C30090FE82E4F090FE817405F002000E787FC2
:1008D300E4F6D8FD75812802032990FE817401F0A6
:1008E30002000E90FE817406F002000E3F065B4F7D
:1008F300666D7D077F6F777C395E79710040761E68
:100903007038375C733E783D6750376EBF86DBCFF8
:10091300E6EDFD87FFEF460102040810204080004A
:0F092300010200030000000400000000000000BB
:00000001FF
